S01700006F70656E626C745F786D63313430302E73726563AD
S31510001000500900201910001000000000991000105F
S3151000101000180400000100001149124A124B00F09A
S3151000102018F8124880471249124A134B00F011F86B
S315100010301249134A134B00F00CF81349134A0020B7
S31510001040521A02DD043A8850FCDC114880471148D8
S3151000105080479B1A03DD043BC858D050FBDC704711
S31510001060642B00100C000020500100207511001098
S31510001070A82C00105009002054090020AC2C001098
S31510001080540900205409002058090020940C00200F
S31510001090BD270010AD270010FEE70000024A936E30
S315100010A001218B439366704700000140004870474A
S315100010B0002D310138B51D4B1B681B041B0E1C4A35
S315100010C0136026D019480268FF211140194C21607F
S315100010D0C26903252A40120211432160C269920592
S315100010E008D49B02C918144800F0C4FA0001134B27
S315100010F018601AE0FFF7DAFF80010D4B19688902B4
S315100011000C4B1B68C91800F0B5FA00010B4B1860A0
S315100011100BE0064BDB699B0503D4094A074B1A60A3
S3151000112003E0FFF7C3FF054B186038BD000301400D
S31510001130580900205C09002000001BB7FC3F002066
S31510001140006CDC0208B50749C0234B62064BD86910
S31510001150064A0240DA61064A1A60C3234B62FFF759
S31510001160A9FF08BD0000014000030140FFFDFFFF7D
S315100011700001F13F08B5FFF791FFFFF7E3FF08BD48
S31510001180034A9188C0239B010B4393807047C04646
S3151000119000000540014B188880B2704700000540DA
S315100011A008B5021C82235B001B68081C111C98479B
S315100011B008BDC04670B5051C0E1C00240BE080232C
S315100011C05B001B68281C9847FFF7E4FFC307FBD496
S315100011D00135FF350134B442F1D370BD08B5102185
S315100011E0FFF7E8FF08BDC04608B5FFF7D9FF08BDF1
S315100011F0F0B54F464646C0B48B08994604339B005B
S315100012001E5803250D40ED00FC27AF40BE431E506F
S31510001210436F4F000326BE40B3434367CB081033DA
S315100012209B001C5807260E40B6000427B740BC4347
S315100012301C501F58BC465778B7403E1C67463E4365
S315100012401E500C4B984204D1036E01268E40B343B8
S31510001250036653688B4043604B4604339B00195812
S315100012601278AA40151C0D431D500CBC9046994689
S31510001270F0BDC04600020440C322014B5A627047BB
S3151000128000000140C022034B5A62024B5B6A5B07A7
S31510001290FBD470470000014010B5041CFFF7F2FFA5
S315100012A0054B1A6914431C61034B1B685B00FBD486
S315100012B0FFF7E2FF10BDC04600030140014B18685E
S315100012C07047C046FC3F0020F0B55F465646C0B496
S315100012D085B083460F1C454B9A4600230293039311
S315100012E001253AE03B689800C0184000291C00F020
S315100012F0C1F901907C68211C00F0BCF9061C0A217A
S3151000130000F0C2F9052905D9301C0A2100F0B2F9FE
S31510001310461C04E0301C0A2100F0ACF9061C002E15
S3151000132006D0B10089194900019800F0A3F904E02C
S3151000133001980A2100F09EF90126A04201D3041B50
S3151000134000E0241A142E07D8A24505D9284B9C4232
S3151000135006D9A246029603950135402DC2D901E061
S3151000136002960395214E0124402512E0681C1F4B5E
S315100013705843029900F07EF93B89834201D8C21A7C
S3151000138000E01A1A964201D9161C2C1C984202D358
S31510001390013D022DEAD8029B191B5B461B684022B1
S315100013A01343584603608B1E1903E023DB011940D3
S315100013B0081C7B89013B9B01FF210B401843071C2E
S315100013C0013C2402F0231B011C402743039B013BD5
S315100013D0C0390B401F435B461F611B6893435A4637
S315100013E0136005B00CBC92469B46F0BD102700005A
S315100013F0E703000010B5E2235B00C4583D33FF330A
S315100014001C42F8D10131120402231A430906114372
S31510001410C333FF33C15010BD10B5041C80208003A8
S31510001420FFF73AFF236801229343236023689B0743
S31510001430FCD410BD10B5E422520083580F24A343E8
S315100014401943815010BDC046E4235B00C058BA3B17
S31510001450FF3B18407047C04608B5FFF7F5FF012857
S3151000146002D0022803D005E0FFF728FF03E0FFF7BC
S315100014701DFE00E0002008BDF0B5474680B4051CEF
S315100014800C1C161CFFF7C8FF281C211CFFF7D2FFE7
S31510001490281CFFF7E1FF041C311C00F0EBF8802735
S315100014A0FF003F1A194B9F4200D91F1C8021C9000B
S315100014B0C91B201C00F0DEF88046B009A409800282
S315100014C0211C00F0D7F8114B984200D9181C444340
S315100014D0A40AA4014346F21A341B002394425B412A
S315100014E0DBB2002B00D0381C002B01D0012300E00A
S315100014F00223E968064A0A40EA60EA689B03184331
S315100015001043E86004BC9046F0BDC046FF030000DF
S31510001510003CFFFF10B5037E012B18D10368202273
S31510001520DA61046821680B4B1940037B1B06F02215
S31510001530120513400B432360036802691A6103689E
S3151000154042695A610368044ADA61002000E0032008
S3151000155010BDC046FFFFFFF04000280010B502681E
S31510001560204BD318990A49039B05DB0E1B020B432C
S3151000157094681D4921409160026891680B439360FD
S31510001580037E012B2CD803682022DA61C3799B06CF
S315100015900ED441684B0F5A078B04134302689361AC
S315100015A081684B0F5A078B0413430268D36005E01A
S315100015B0036842689A6103688268DA60041C037ED5
S315100015C0012B06D1FFF7A6FF236880221205DA61E8
S315100015D003E0036880221201DA612368034ADA61A4
S315100015E010BDC04600F0FBAFFF00FFFF4000A00695
S315100015F00268D169D369DB05DB0F890606D5012B95
S3151000160006D0E023DB04D361002002E0042000E0D2
S31510001610022070470268D169D3695B07DB0F0905A1
S315100016200FD4012B0FD01369036153694361D1693C
S31510001630D3691B07DB0F490707D5002BF3D1002011
S3151000164004E0032002E0022000E000207047C046BC
S3151000165030B58B0804339B001C5803252940C9005C
S31510001660F9358D40AC431C501C588A40111C21433F
S31510001670195030BD034B04225A6318625962986A96
S315100016807047C04600000340034B04225A63186299
S315100016905962D96A986A70470000034070B5051CF4
S315100016A00E1C00F0EFF8F479002C00D11034281C31
S315100016B03168221C00F050F8B379013B5B006408D6
S315100016C0013424021C43114B1C43EC633379013B58
S315100016D01B068122520013436B637379002B05D0CE
S315100016E06A6B013B1B0413436B6305E0696B32792C
S315100016F0531E1B040B436B63A023DB00AB63012358
S315100017005B42EB6433892B6470BDC0460100030055
S3151000171084235B00C258E023DB041A4208D1836B92
S315100017201B06FCD480239B01C3648023C15002E0B6
S31510001730C0235B00C150704786235B00C258E0236C
S31510001740DB041A4202D1406D80B203E08E235B00A7
S31510001750C05880B27047C046F0B55F464E46C0B41A
S3151000176083B063293DD9002A3DD0151C0C1C834635
S31510001770FFF7A4FD6421FFF77DFF8146201C64213D
S31510001780FFF778FF071C1B4E012301930093341CAF
S3151000179011E048466043291C7943FFF76BFF830A23
S315100017A08005800D134A934204D8B04202D2061C1B
S315100017B001930094013C002CEBD180231B02009F67
S315100017C01F435B461F615A690B4B1340013DAD0227
S315100017D01D43019E013E360435435B465D61002084
S315100017E002E0012000E0012003B00CBC91469B46AC
S315100017F0F0BDC046FF030000EF8000FC70B58425E5
S315100018006D004659064C344044514659054C264005
S315100018101B02194314060A1C22433243425170BD5F
S31510001820FFFFFFF8C0C0FFF870B586256D0046595A
S31510001830084C344044514659074C26401B02194364
S3151000184014060A1C22433243802149050A43425199
S3151000185070BDC046FFFFFFF8C0C0FFEF08B5074BCD
S31510001860984203D10820FFF717FD06E0044B984273
S3151000187003D18020C002FFF70FFD08BD0800004805
S315100018800840004810B5041C9023DB05984202D08E
S315100018900C4B984203D10C48FFF7E0FF08E00B4BC6
S315100018A0984202D00A4B984202D10A48FFF7D6FF57
S315100018B00323E360E368DB07FCD5236C0F22934315
S315100018C0236410BD0002004808000048004000488C
S315100018D000420048084000487047C04672B670473C
S315100018E062B6704730B585B0FFF7E8FC041C00E01F
S315100018F064004D4B9C42FBD900E064084B4B9C4264
S31510001900FBD84B480121221CFFF7B6FD01A9019413
S31510001910484B4B60FA235B010B8101254D81464CE8
S31510001920201CFFF7D1FC2268402313432360236851
S315100019301D432560414A42481060D3793F210B4030
S31510001940BF390B43D37153685B0F5B073D4C234381
S3151000195053609168490F4907214391601B0E20245B
S31510001960A343D371090E20231943D172C368802172
S3151000197089050B43C36008231373002305E02F4A20
S31510001980D218002111740133DBB2072BF7D92B487B
S3151000199001230376FFF7E2FD254801210022FFF718
S315100019A029FD294A29481060D3793F210B40BF39B8
S315100019B00B43D37153685B0F5B07254C234353606E
S315100019C09168490F4907214391601B0E2024A343B8
S315100019D0D371090E20231943D172C368802189055A
S315100019E00B43C36008231373002305E0164AD2186D
S315100019F0002111740133DBB2072BF7D912480023EB
S31510001A000376FFF7ABFD0A4801210122FFF7F2FC2E
S31510001A10094B1A6840218A431A601A683F398A436B
S31510001A201A6005B030BDC046FF1AB700000E270772
S31510001A300000045020A10700000304506009002094
S31510001A4000100450E1070000800900202010045007
S31510001A506706000010B50F4B1973002305E0C45C30
S31510001A600C4AD21814740133DBB28B42F7D3094CEB
S31510001A70201CFFF74FFD23680222DA61201CFFF7B6
S31510001A80B7FD01E000F010FC024B1B68DB699B07F9
S31510001A90F8D410BD6009002010B5114B1B68DB6926
S31510001AA0DB071AD5041C0E48FFF7B4FD002809D031
S31510001AB000200DE00A4AD218127CE2540133DBB240
S31510001AC0012001E000200023054A127B9A42F1D83A
S31510001AD0034B1B680122DA6100E0002010BDC046EE
S31510001AE08009002008B5FFF7F9FE08BD10B500F013
S31510001AF00FFA00280DD000F0C7FD002809D000F01D
S31510001B008DFB00F015FA00F007FA4468FFF7E8FEBF
S31510001B10A04710BD70B508E0461C4D1C0B7803702D
S31510001B2000F0C2FB221C301C291C531E9CB2002A3A
S31510001B30F2D170BD38B5051C002419E000F0B4FBD5
S31510001B4063001B199B000C495958A9420ED8630013
S31510001B501B199B000848C3185B68C918A94205D908
S31510001B6063001A1992008218107A04E00134E4B264
S31510001B702F2CE3D9FF2038BD0828001038B5051CD6
S31510001B80002410E000F090FB63001B199B00084A2C
S31510001B90D3181B7AAB4204D16300191989008858EF
S31510001BA005E00134E4B22F2CECD90120404238BDB7
S31510001BB00828001008B5FF230B4209D103688B4291
S31510001BC008D002C080225200FFF7A4FF012002E0D5
S31510001BD0002000E0012008BD38B5041C0068FFF79E
S31510001BE0A9FFFF2826D0FFF7CBFA00F0C9F9451D4B
S31510001BF0211C01C9FFF7F8FA05E000F0C1F9A84267
S31510001C001AD800F051FBFFF7C5FAC307F5D4FFF752
S31510001C10C1FA002812D1002308E02268D2181278DF
S31510001C20D2B2E11809798A420AD10133FF2BF4D9CD
S31510001C30012006E0002004E0002002E0002000E081
S31510001C40002038BD38B5041C0D1C0C4B984207D02B
S31510001C500B4B994206D0FFF7BFFF002803D109E0CE
S31510001C60084C00E0054C201C291CFFF7A3FF002898
S31510001C7002D102E0002000E0201C38BDA00900209F
S31510001C8000300010A40A0020F0B5474680B4071CA7
S31510001C900C1C151C1E1C0B0A1B02984603680133EC
S31510001CA004D14146FFF786FF002827D03B684345FD
S31510001CB005D0381C4146FFF7C5FF071E1BD03B68F1
S31510001CC0E41A3C19043400F0EFFA3B1DE31AFF2B1B
S31510001CD008D94346591CFF31381CFFF7B3FF071EBE
S31510001CE00BD0041D2B78237001340135013E002ED4
S31510001CF0E9D1012002E0002000E0002004BC90465B
S31510001D00F0BDC046F8B5051C0F1C88422AD802281B
S31510001D102AD9322922D929E000F0C6FA281CFFF761
S31510001D202DFF061C431C23D0FFF72AFA00F028F9D2
S31510001D300A30041C301CFFF751FA05E000F020F9B8
S31510001D40A04217D800F0B0FAFFF724FAC307F5D46B
S31510001D50FFF720FA00280FD10135EDB2BD42DBD9CD
S31510001D6001200AE0002008E0002006E0002004E040
S31510001D70002002E0002000E00020F8BD01235B42B5
S31510001D80024A1360024A13607047C046A40A002034
S31510001D90A009002070B5041C0D1C161CFFF7CAFE06
S31510001DA0FF2818D060190138FFF7C4FEFF2814D099
S31510001DB0230A1B020A4A934206D10A48211C321CE6
S31510001DC02B1CFFF761FF09E00748211C321C2B1C56
S31510001DD0FFF75AFF02E0002000E0002070BDC04669
S31510001DE000300010A0090020A40A0020F8B5061C37
S31510001DF00C1CFFF79FFE051C30190138FFF79AFEE1
S31510001E00011CFF2D05D0FF2805D0281CFFF77AFFEF
S31510001E1002E0002000E00020F8BDC04600B583B007
S31510001E200F4B1B68013318D00D4B5A6898688446BF
S31510001E306244111CDA68944661441A6994466144F6
S31510001E405A69944661449A698B185B420193054816
S31510001E50042101AAFFF79EFF00E0012003B000BD98
S31510001E60A0090020183000100C4B1A680C4B1B6888
S31510001E70D3180C4A1268D3180B4A1268D3180B4A97
S31510001E801268D3180A4A1268D3180A4A1268D31865
S31510001E90002B01D1012000E0002070470030001017
S31510001EA004300010083000100C30001010300010F4
S31510001EB0143000101830001008B50B4B1B68013396
S31510001EC004D00948FFF788FE00280CD0074B1B6882
S31510001ED0013305D00548FFF77FFE002802D102E046
S31510001EE0012000E0012008BDA0090020A40A00205E
S31510001EF0004870470030001008B5FFF73FFF08BDD7
S31510001F0008B5FFF747FF08BD08B5FFF76FFF08BD17
S31510001F1008B5FFF7A9FF08BD08B5FFF7E9FF08BD2B
S31510001F2008B5FFF77BFF002801D0FFF7C5FF08BDF6
S31510001F300022014B1A60704710E000E008B5FFF769
S31510001F40F7FF054B054A5A6000229A600521196071
S31510001F50034B1A6008BDC04610E000E07FBB0000CE
S31510001F60A80B0020044B1B68DB0303D5034A136838
S31510001F70013313607047C04610E000E0A80B002044
S31510001F8008B5FFF7EFFF014B186808BDA80B002036
S31510001F9008B58A235B000B4AD358DB0410D481B2F0
S31510001FA0101CFFF7B5FB8A235B00064AD358DB05E6
S31510001FB0F9D5802149008C235B00D150012000E027
S31510001FC0002008BD0002004810B58A235B00064AAF
S31510001FD0D3581B0706D4041C101CFFF7ADFB20704A
S31510001FE0012000E0002010BD0002004810B584B0AA
S31510001FF001A9E1231B02019308230B714B71073BC7
S315100020008B710F33CB7100230B810C4C201CFFF707
S3151000201045FB201C102104220123FFF7EFFB201C97
S31510002020002104220123FFF7FFFB236C0F229343A9
S315100020300D3A1343236404B010BDC0460002004895
S3151000204070B5061C0D1E402D03D91048752100F0E1
S3151000205071F8281CFFF79CFF012803D00B48792143
S3151000206000F068F800240CE000F01EF9305DFFF770
S315100020708FFF012803D00548822100F05BF8013458
S31510002080A4B2ABB2A342EFD870BDC046482A001026
S3151000209038B5051C234B1C78002C13D12248FFF7AA
S315100020A093FF01283CD1204B1B78002B33D0FFF730
S315100020B067FF1E4B186000221D4B1A700132194B18
S315100020C01A702DE01A4B18780130174B1818FFF7B5
S315100020D07BFF041E012C12D1154B1A780132D2B295
S315100020E01A70114B1B789A4217D192B2281C0E49BE
S315100020F00131FFF70FFD00220A4B1A7010E0FFF7AF
S315100021003FFF0A4B1B686433984208D90022054BDF
S315100021101A70002404E01C1C02E0002400E00024D5
S31510002120201C38BDF10B0020AC0B0020F40B002056
S31510002130F00B002008B500F0B7F8FCE708B500F082
S31510002140ABF8012810D0094B1B78012B0CD1FFF7E7
S3151000215017FF074B1B68F533FF33984204D3002251
S31510002160024B1A70FFF7C2FC08BDC046F80B0020E0
S31510002170FC0B002008B50122044B1A70FFF700FF74
S31510002180034B1860FFF7DAFF08BDC046F80B0020B6
S31510002190FC0B002008B5FFF7A5FC00F081F8FFF74F
S315100021A0CDFEFFF7A9FE00F00DF8FFF7E3FF08BD1F
S315100021B008B500F079F8FFF7D5FE00F013F8FFF731
S315100021C0BDFF08BD10B500F0E5F9FFF78BFB044C19
S315100021D001232370FFF70AFF0023237010BDC046AA
S315100021E05009002008B50B48FFF756FC012805D109
S315100021F00122094B1A70074800F0EAF90548FFF763
S3151000220047FF012805D10022034B1A70014800F040
S31510002210DFF908BD000C0020500900207047C046A9
S3151000222038B5051C0C1C094B1B78012B02D1C9B201
S31510002230FFF710FC054B1B78002B03D1E1B2281CCD
S31510002240FFF7FEFE00F0BCF938BDC046500900206D
S31510002250074B1B78022B05D0032B05D0012B05D07D
S31510002260402004E0002002E0002000E00820704733
S3151000227050090020074B1B78022B05D0032B05D0E5
S31510002280012B05D0402004E0002002E0002000E0F1
S31510002290082070475009002008B500F089F908BDDC
S315100022A008B500F0F7F908BD08B500F0F9F908BD52
S315100022B010B5002304E00178CB18DBB20130211CE5
S315100022C04C1E0029F7D11360012010BD0022014BCE
S315100022D05A707047400C0020034BFE22DA701871BA
S315100022E00221BA3A99527047400C002010B5054C9D
S315100022F000232370FFF7EAFFFF23E3700122BB3BA5
S31510002300E25210BD400C0020064BFF22DA7000226C
S315100023101A71597859719A71DA711A720621443202
S3151000232099527047400C002008B50020FFF7D4FFE3
S3151000233008BDC046094BFF22DA70094A9A6400228A
S315100023401A715A719A710721D9710021197259722D
S3151000235099720831442299527047C046400C0020A9
S315100023605C2B0010044BFF22DA7042689A6401213C
S31510002370442299527047C046400C002010B5084CB4
S31510002380FF23E3704168E21DA06CFFF791FF2071F7
S3151000239000236371A37108224433E25210BDC04674
S315100023A0400C002008B53120FFF796FF08BDC04647
S315100023B038B5084CFF23E370002525716571FFF7CA
S315100023C047FFA071E5712572657207224423E25218
S315100023D038BDC046400C002038B5FFF777FF0D4CCE
S315100023E001252570FF23E370EF3B237100236371F2
S315100023F0FFF72EFFA071FFF73DFFE071FFF73AFFE1
S31510002400000A20726572A57208224423E252FFF771
S3151000241073FD38BD400C002038B5051C4478FFF715
S3151000242017FF0138844203DD2220FFF755FF10E025
S31510002430084C201D6A78A16CFFF76CFBFF23E37034
S315100024406B78A26C94466344A3646B780133442280
S31510002450A35238BD400C002038B5041C4578FFF750
S31510002460F7FE0138854203DD2220FFF735FF11E024
S315100024706168094DA964281D6278FFF74BFBFF239D
S31510002480EB706378AA6C94466344AB64637801334B
S315100024904422AB5238BDC046400C002038B5041C4F
S315100024A00E4B9D6CFFF7D4FE411E621C281CFFF7D5
S315100024B027FD002803D13130FFF70EFF0CE0074C43
S315100024C0FF23E370FFF7C4FE0138A36C9C466044FB
S315100024D0A06401224423E25238BDC046400C0020BD
S315100024E038B5041C4578FFF7B3FE0238854203DD84
S315100024F02220FFF7F1FE21E0114BFF22DA700121B5
S31510002500BB3A99526178002907D1FFF709FD0028D7
S3151000251014D13130FFF7E0FE10E0094B986CA21C85
S31510002520FFF7EEFC002803D13130FFF7D5FE05E0AA
S315100025306378034A916C8C466344936438BDC046F5
S31510002540400C002008B5094B9B6C4168181CFFF71E
S31510002550DBFC002803D13130FFF7BEFE05E0034B4C
S31510002560FF22DA700121BB3A995208BD400C0020B7
S3151000257008B5FFF7BBFA034BFF22DA700121BB3A0D
S31510002580995208BD400C002008B589B2FFF748FEE5
S3151000259008BDC046054B00221A709A6443215A544E
S315100025A001315A529A705A707047C046400C00203A
S315100025B0024B1878002800D001207047400C0020EC
S315100025C000214323014AD1547047C046400C0020D5
S315100025D008B50378FF2B02D1FFF7FEFE38E0284A34
S315100025E01278012A4AD13733DAB2352A2DD8930018
S315100025F0244AD3589F46FFF70FFF29E0FFF72CFF19
S3151000260026E0FFF7AFFE23E0FFF7B8FE20E0FFF766
S3151000261091FE1DE0FFF788FE1AE0FFF775FE17E042
S31510002620FFF764FE14E0FFF739FF11E0FFF758FFDC
S315100026300EE0FFF7BDFE0BE0FFF784FF08E0FFF7A3
S3151000264097FF05E0FFF7AEFE02E02020FFF744FEFD
S3151000265043230B4AD35C012B02D11020FFF73CFE1B
S315100026604423074AD15A0BB2002B07DD101C012256
S315100026704323C254033009B2FFF786FF08BDC04694
S31510002680400C0020842A001008B500F049F80120FB
S3151000269008BDC04608B5642000F006F808BDC0465F
S315100026A008B500F013F808BD38B5051C054C201CFC
S315100026B000218022FEF7CCFF01236360024B1D80B0
S315100026C038BDC046000404408E0C002008B5FFF744
S315100026D057FC0F4B1B68984218D30E4B1B78002BD8
S315100026E007D101220B4B1A70802252020A4B5A60F4
S315100026F005E00022074B1A700132074B5A60FFF7AC
S315100027003FFC064B1B88C018014B186008BDC0461D
S31510002710900C00208C0C0020000404408E0C00202D
S315100027200122014B5A6070470004044030B589B04D
S3151000273006AA00251570194C201C0321FEF758FD1A
S3151000274004AA9C231370201C0221FEF751FD144B82
S31510002750DA6950218A43DA61DA690724A243DA6119
S3151000276002AA15700F4D281C4839FEF741FDA42307
S315100027706A461370281C0921FEF73AFD0A4B1A689F
S31510002780402002431A60DA68A24302210A43DA6043
S315100027901A6882431A6009B030BDC0460001044071
S315100027A000020048000404400003045008B5FFF777
S315100027B0F1FCFFF7BBFFFFF7FBFCFCE70E4B70B518
S315100027C000251E1C0D4CE41AA410A54204D0AB0023
S315100027D0F35898470135F8E7FFF77EF8084B0025C0
S315100027E01E1C084CE41AA410A54204D0AB00F358E2
S315100027F098470135F8E770BD5409002054090020A8
S315100028005409002054090020003000100010000068
S31510002810030000000040001000100000040000003B
S3151000282000500010001000000500000000600010AD
S3151000283000100000060000000070001000100000DC
S3151000284007000000008000100010000008000000C3
S3151000285000900010001000000900000000A00010F9
S31510002860001000000A00000000B000100010000068
S315100028700B00000000C00010001000000C0000004B
S3151000288000D00010001000000D00000000E0001045
S31510002890001000000E00000000F0001000100000F4
S315100028A00F000000000001100010000010000000D2
S315100028B0001001100010000011000000002001108F
S315100028C0001000001200000000300110001000007F
S315100028D0130000000040011000100000140000005A
S315100028E000500110001000001500000000600110DB
S315100028F0001000001600000000700110001000000B
S3151000290017000000008001100010000018000000E1
S3151000291000900110001000001900000000A0011026
S31510002920001000001A00000000B001100010000096
S315100029301B00000000C00110001000001C00000069
S3151000294000D00110001000001D00000000E0011072
S31510002950001000001E00000000F001100010000022
S315100029601F000000000002100010000020000000F0
S3151000297000100210001000002100000000200210BC
S3151000298000100000220000000030021000100000AD
S315100029902300000000400210001000002400000078
S315100029A00050021000100000250000000060021008
S315100029B00010000026000000007002100010000039
S315100029C02700000000800210001000002800000000
S315100029D000900210001000002900000000A0021054
S315100029E0001000002A00000000B0021000100000C5
S315100029F02B00000000C00210001000002C00000088
S31510002A0000D00210001000002D00000000E002109F
S31510002A10001000002E00000000F002100010000050
S31510002A202F0000000000031000100000300000000E
S31510002A3000100310001000003100000000200310E9
S31510002A400010000032000000433A2F576F726B2FB0
S31510002A50736F6674776172652F4F70656E424C5452
S31510002A602F5461726765742F536F757263652F41AA
S31510002A70524D434D305F584D43312F756172742E50
S31510002A8063000000262600104A2600104A26001071
S31510002A90442600104A2600104A2600103E26001032
S31510002AA02C26001038260010322600104A26001058
S31510002AB04A2600104A2600104A2600104A26001000
S31510002AC04A2600104A2600104A2600104A260010F0
S31510002AD04A2600104A2600104A2600104A260010E0
S31510002AE04A2600104A2600104A2600104A260010D0
S31510002AF04A2600104A2600104A2600104A260010C0
S31510002B004A2600104A2600104A2600104A260010AF
S31510002B104A2600104A2600104A2600104A2600109F
S31510002B204A2600104A2600104A26001008260010D1
S31510002B30FC250010F6250010022600104A2600106B
S31510002B404A2600104A2600100E2600104A260010AB
S31510002B50142600101A260010202600104F70656EDD
S30910002B60424C540079
S31510002B642C48004700000000000000000000000090
S31510002B74000000000000000000000000000000003B
S31510002B8425480047000000000000000023480047C5
S31510002B942348004723480047234800472348004753
S31510002BA42348004723480047234800472348004743
S31510002BB42348004723480047234800472348004733
S31510002BC42348004723480047234800472348004723
S31510002BD42348004723480047234800472348004713
S31510002BE42348004723480047234800472348004703
S31510002BF423480047234800472348004723480047F3
S31510002C0423480047234800472348004723480047E2
S31510002C1423480047991000109910001099100010BD
S31510002C2499100010991000109910001099100010A6
S31510002C349910001099100010991000109910001096
S31510002C449910001099100010991000109910001086
S31510002C549910001099100010991000109910001076
S31510002C649910001099100010991000109910001066
S31510002C749910001099100010991000109910001056
S31510002C849910001099100010991000109910001046
S31510002C949910001099100010991000109910001036
S30910002CA4991000105D
S30910002CA8040000000E
S70510001019C1
